:100000000C94D1010C9415020C9415020C94150259
:100010000C9415020C9415020C9415020C94150204
:100020000C9415020C9415020C941E0D0C94F00DFA
:100030000C9415020C9415020C9415020C941502E4
:100040000C9415020C945A200C9415020C94150271
:100050000C9415020C943C1B0C9415020C94150284
:100060000C9415020C9415020C9415020C941502B4
:100070000C9415020C9415020C9415020C941502A4
:100080000C9415020C9415020C9415020C94150294
:100090000C9415020C9415020C9415020C94150284
:1000A0000C9415020C9415020C9415025D0E7F0E33
:1000B0006D0F7F0E6D0FC40EE70E6D0F3C0F4F0FCF
:1000C0001E121E124D124D128312A312D413D413FA
:1000D000AE12D4135E135E13C513D413D413CE1310
:1000E0006B136B136B136B136B136B136B136B1320
:1000F0006B136B136B136B136B136B136B136B1310
:100100007D138A1391139813A21335002B002961D4
:10011000E1003A0000001E00140004001D003B0036
:10012000E2001F001A0016001B003C00296120009D
:100130000700080006003D002A0021000900170002
:100140001900E300A90022000E000A0005000000CB
:10015000AA003E00310000002F000000A8003F0070
:100160000000000030000000AE0023000D001C0065
:1001700013000000AB002400180011001000E7007D
:10018000AC00250015000C00360050002C002600A5
:100190000F001200370051003400270033000B001D
:1001A00038005200E6002E002D002800E5004F0028
:1001B000000016034500720067006F0044006F00E6
:1001C0007800200045005A00000016034500720028
:1001D00067006F0044006F007800200045005A005F
:1001E00000000403090409026D00040100A0FA09DB
:1001F0000400000103010100092111010001224056
:10020000000705810308000A090401000103010237
:1002100000092111010001224D0007058203080099
:100220000A09040200010300000009211101000174
:100230002236000705830308000A090403000103AE
:100240000000000921110100012239000705840383
:100250001000011201100100000008EDFE0713015B
:10026000000102000105010906A101050719E029A5
:10027000E715002501950875018102050819012976
:100280000595057501910295017503910105071901
:1002900000297715002501957875018102C00501B7
:1002A0000980A101850216010026B7001A01002A63
:1002B000B700751095018100C0050C0901A10185E9
:1002C00003160100269C021A01002A9C0275109553
:1002D000018100C005010902A1010901A100050970
:1002E0001901290515002501950575018102950162
:1002F000750381010501093009311581257F9502BA
:100300007508810609381581257F950175088106D4
:10031000050C0A38021581257F950175088106C0F4
:10032000C005010906A101050719E029E715002507
:10033000019508750181029501750881010508196B
:100340000129059505750191029501750391010536
:1003500007190029FF150026FF0095067508810082
:10036000C0000000000000000000000001020406C0
:100370000A0F17202C3A4A5D71879DB3C7DAE9F559
:10038000FCFFFCF5E9DAC7B39D87715D4A3A2C2082
:10039000170F0A0604020100000000000000000020
:1003A000000011241FBECFEFDAE0DEBFCDBF04B6E0
:1003B00003FE24C08091FD019091FE01A091FF01F8
:1003C000B09100028730904BA740B04BB9F4109227
:1003D000FD011092FE011092FF011092000214BE66
:1003E00084B7877F84BF88E10FB6F894809360005C
:1003F000109260000FBEE0E0FFE3099511E0A0E07D
:10040000B1E0E2E4F4E402C005900D92A433B10738
:10041000D9F711E0A4E3B1E001C01D92AD3FB107EF
:10042000E1F70E94660A0C941F220C9400001092BF
:10043000B9008AE08093B800089594EA9093BC00D4
:100440009091BC0097FFFCCF9091B900987F9830B5
:1004500021F0903111F081E008958093BB0084E891
:100460008093BC008091BC0087FFFCCF8091B900D5
:10047000887F883111F0803471F780E0089584E935
:100480008093BC008091BC0084FDFCCF08958093D4
:10049000BB0084E88093BC008091BC0087FFFCCF48
:1004A0009091B900987F81E0983209F480E0089536
:1004B00084E88093BC008091BC0087FFFCCF8091D2
:1004C000BB00089580B38C7080BB81B3836F81BB08
:1004D000089580910101811115C080E40E941D02E0
:1004E0008093010181110CC082E10E944702809338
:1004F0000101811105C08FEF0E9447028093010125
:100500000E943F0284B1807F84B985B1807F85B924
:100510008AB1837F8AB98BB1837F8BB93E98469825
:1005200008950E943304809301010E9469020E9491
:100530006202A5E3B1E0E3E4F1E08EE08E0F1192F8
:100540001D928E13FCCF0C941D040E9433048093E3
:1005500001010E9469020E946202A5E3B1E0E3E4A6
:10056000F1E08EE08E0F11921D928E13FCCF089554
:10057000BF92CF92DF92EF92FF920F931F93CF9390
:10058000DF9380910101882379F0809134018F5F9E
:1005900080933401811108C00E94330480930101CB
:1005A000811102C00E94C50305E311E0C0E0D0E064
:1005B000DD24D39482E0C82EEE24E394F12CC730DE
:1005C000D10500F580910101811164C080E40E9491
:1005D0001D0280930101811112C082E10E94470235
:1005E0008093010181110BC0C7010C2E01C0880F3F
:1005F0000A94EAF780950E944702809301010E94C5
:100600003F0248C0CA30A1F028F4C83059F0C930C0
:1006100061F005C0CC3089F070F0CD3089F0209ABF
:10062000289810C0219A29980DC0229A2A980AC0A9
:10063000239A2B9807C0529A01C0539A5B9802C024
:100640003E9A469890EA9A95F1F79FB1799902C03F
:1006500082E001C080E091709D25982B7C9902C0BA
:1006600084E001C080E0892B7D9902C038E001C0A0
:1006700030E0832B7E9902C020E101C020E0822B74
:100680009FB19095991F9927991F9295990F907EE8
:10069000892B0FC080910101811149C080E40E9423
:1006A0001D0280930101882379F1B12C0E943F0241
:1006B0008B2DF8019081981719F08083C09200016A
:1006C0000E94690221960F5F1F4FCE30D10509F0BD
:1006D00076CF80910001882361F1815080930001E1
:1006E000882339F08FE99FE00197F1F700C00000FF
:1006F00020C0A3E4B1E0E5E3F1E0CF01825F919196
:100700009D938E13FCCF15C083E10E944702809316
:1007100001018111CACF81E40E941D028093010171
:100720008111C3CF0E945802B82EB094BFCF80E091
:10073000C0CF0E94C30381E0DF91CF911F910F9141
:10074000FF90EF90DF90CF90BF900895E82FF0E0FA
:10075000ED5BFE4F8081089508950F931F93CF9313
:10076000DF93C3E4D1E010E00C2F025F899190E0A9
:100770000E94B31A180F0C13F9CF812FDF91CF917C
:100780001F910F9108950C948E0456985E982598A9
:100790002D9826982E9827982F988FEF90E0909379
:1007A00089008093880090938B0080938A009093B7
:1007B0008D0080938C00259A2D9A2FEF80E792E090
:1007C000215080409040E1F700C00000269A2E9A08
:1007D0002FEF80E792E0215080409040E1F700C089
:1007E0000000279A2F9A2FEF80E792E02150804057
:1007F0009040E1F700C0000025982D982FEF80E78A
:1008000092E0215080409040E1F700C0000026981F
:100810002E982FEF80E792E0215080409040E1F742
:1008200000C0000027982F9856985E9825982D981C
:1008300026982E9827982F98089589EA809380000B
:1008400089E08093810024982C983F988AB18F7416
:100850008AB96E98479A8BB1806B8BB9769A0E9451
:10086000C5030C94850480E28093010180915101BD
:1008700081110EC00E94170281E0809351012FEF79
:1008800083ED90E3215080409040E1F700C00000EC
:1008900080E40E941D028093010181112EC00E94FC
:1008A000470280930101811128C00E944702809372
:1008B0000101811122C08FE30E9447028093010150
:1008C00081111BC00E943F0280E40E941D028093A0
:1008D0000101811112C08CE00E9447028093010146
:1008E00081110BC00E94470280930101811105C054
:1008F0008FE30E944702809301010E943F02809192
:100900000101089580E090E0089556985E9825983A
:100910002D9826982E9827982F980895089581E06D
:10092000089581E008950C9491040895282F882358
:1009300039F090E02A3010F44D9608950697089506
:1009400087E290E00895AF92BF92DF92EF92FF921C
:100950000F931F93CF93DF938C01FC01C081D18152
:10096000CE010E943819BE010E941308EC01B801A3
:100970000E949304882309F4C9C1F8018281882365
:1009800009F4BEC080915E0181111FC0C431F0E73F
:10099000DF0709F0B5C10E94950481E080935E01F4
:1009A0000E94061B90935D0180935C01109255019B
:1009B000109257011092560110925901109258014D
:1009C00010925B0110925A01A1C180915C0190913B
:1009D0005D010E94121B883C910570F480915501C5
:1009E000E82FF0E0EE0FFF1FEA5AFE4FD183C083DD
:1009F0008F5F809355018AC1C13020E8D20708F487
:100A000051C0F8018281882309F47EC05E01E89418
:100A1000B7F880915401813079F050F08230C1F400
:100A200082EE0E94C21087E50E94C21087E50EC0C8
:100A300082EE0E94C2100CC080EE0E94C21081EEB5
:100A40000E94C21088E10E94C21088E10E948A11AF
:100A50008CE0E82EF12CC5010E2C02C096958795EE
:100A60000A94E2F78F700E949604D82E0E94C2105A
:100A70008D2D0E948A11F4E0EF1AF1082CEFE21696
:100A80002FEFF20641F780915401813029F010F0E8
:100A9000823041F482EE04C080EE0E948A1181EE21
:100AA0000E948A11C43180E7D80768F4C23090E709
:100AB000D90708F046C0C115E0E7DE0771F0C13084
:100AC000D047A1F10CC1C33320E7D20709F4D8C045
:100AD000C433D04709F4EBC002C1F80182818823F6
:100AE00009F402C10E943F14FFEF24E38CE0F150AF
:100AF00020408040E1F700C000000E94611B06C159
:100B0000C13080E8D80770F2C43120E7D20708F07E
:100B1000B3C0C23080E7D807A0F4C11590E7D90769
:100B200009F4E2C0C130D04709F0D9C0F801828190
:100B3000882309F4D9C08091DB0181608093DB01B7
:100B4000E5C0F8018281882309F4CEC00E94BB1B56
:100B5000811102C00E94A11B0E94CE1B90E09093C5
:100B6000EF018093EE01C230F0E7DF0721F48091BE
:100B7000EE0181607AC0C33020E7D20721F4809172
:100B8000EE01826072C0C43080E7D80721F4809102
:100B9000EE0184606AC0C53090E7D90719F48091EE
:100BA000EE0127C0C630E0E7DE0721F48091EE01B8
:100BB00080615BC0C730F0E7DF0721F48091EE0170
:100BC000806253C0C83020E7D20721F48091EE0143
:100BD00080644BC0C93080E7D80721F48091EE01D2
:100BE000806843C0CA3090E7D90729F48091EE01AC
:100BF000846088603AC0CB30E0E7DE0721F4809162
:100C0000EE018E7F32C0CC30F0E7DF0721F4809117
:100C1000EE018D7F2AC0CD3020E7D20721F48091EC
:100C2000EE018B7F22C0CE3080E7D80719F4809187
:100C3000EE011AC08091EE01CF3090E7D90711F490
:100C40008F7E13C0C031E0E7DE0711F48F7D0DC049
:100C5000C131F0E7DF0711F48F7B07C0C231D04705
:100C600011F48F7702C08B7F877F8093EE01809194
:100C7000EE010E94D21B4AC0C333F0E7DF07A1F4A4
:100C8000F8018281882321F01092520182E016C07F
:100C900080915201811106C086E20E94C21086E254
:100CA0000E948A1182E018C0C433D047C1F4F80111
:100CB0008281882331F01092530180E20E94D91181
:100CC00025C080915301811106C087E20E94C210A5
:100CD00087E20E948A1180E20E94E01117C081E041
:100CE0008093520180935301C801DF91CF911F91EE
:100CF0000F91FF90EF90DF90BF90AF900C948F0416
:100D0000C130F0E8DF0708F081CECCCE80E0DF9183
:100D1000CF911F910F91FF90EF90DF90BF90AF9018
:100D2000089526E0729FF001112444E5849FE00DB0
:100D3000F11D1124E60FF11DEE0FFF1FE65FFE4FC0
:100D4000859194910E942508811560E49607B0F57D
:100D5000811570E3970708F0DEC0803E9105D8F456
:100D6000803C910508F06CC0883A910578F4853A8A
:100D7000910508F06BC08130910509F452C108F467
:100D80000FC18430910508F04CC10AC18B3B91051D
:100D900008F467C005C18F3F910509F048F4803F12
:100DA000910508F0ADC0883E910508F43AC1F8C03D
:100DB000811520E2920708F0A5C00895811543E54A
:100DC000940790F4811562E5960708F0C8C0811574
:100DD00071E5970708F0BEC0811520E5920708F07D
:100DE0009DC09F70906A0895811545E59407D8F4D9
:100DF000811564E5960708F0C8C0482F46954695CA
:100E000070E2479FA00111248370992721E030E010
:100E1000B90102C0660F771F8A95E2F7CB01842BD8
:100E2000952B9A680895811576E5970708F4B2C066
:100E30009C0130562115304108F0B2C09F70AEC001
:100E4000FC01EE0FFF1FE657F04062C0853A9105A6
:100E500009F4A9C0863A910509F0A8C082E890E497
:100E60000895883A910509F4A4C0893A910509F4D6
:100E7000A3C08A3A910509F4A2C08B3A910509F4FE
:100E8000A1C08C3A910509F4A0C08D3A910509F4EE
:100E90009FC0803B910509F49EC08E3A910509F4EC
:100EA0009DC08F3A910509F49CC0813B910509F4DE
:100EB0009BC0823B910509F49AC0833B910509F4DC
:100EC00099C0843B910509F498C0853B910509F4CC
:100ED00097C0863B910509F496C0873B910509F4BC
:100EE00095C0883B910509F494C0893B910509F4AC
:100EF00093C08A3B910509F492C080E094E4089580
:100F000090650895FC01FF70EE0FFF1FE65FFE4F36
:100F10008591949108959927906C0895482F437076
:100F200021E030E002C0220F331F4A95E2F73C680F
:100F3000AC0164E0569547956A95E1F74370342B10
:100F40008F708695869560E2869FC0011124822B62
:100F5000932B0895982F8827816F906A0895482FC2
:100F60004695469570E2479FA0011124837099270A
:100F700021E030E0B90102C0660F771F8A95E2F7E1
:100F8000CB01842B952B9C680895982F8827846F1C
:100F9000906A08958F719927982F882790620895F5
:100FA00080E090E0089581E890E4089583E890E47B
:100FB000089582EE94E4089589EE94E408958AEE0B
:100FC00094E4089585EB94E4089586EB94E4089501
:100FD00087EB94E408958CEC94E408958DEC94E40C
:100FE000089583E895E408958AE895E4089582E9F0
:100FF00095E4089584E995E4089581E296E40895DE
:1010000083E296E4089584E296E4089585E296E406
:10101000089586E296E4089587E296E408958AE2C8
:1010200096E40895089596E0799FF001112494E5DF
:10103000899FE00DF11D1124E60FF11DEE0FFF1F3A
:10104000E65FFE4F8591949108958238910549F1AC
:10105000B0F48133910509F458C048F48932910500
:1010600009F44EC08A32910509F454C008958533BD
:10107000910509F440C08933910599F00895833EA4
:10108000910529F138F4803E910591F0823E910559
:10109000A1F00895863E9105F9F0873E910531F162
:1010A00008952091EE0120FD3AC021FD38C0089539
:1010B0008091EE0180FD35C032C08091EE0182FF4B
:1010C00032C08091EE0184FD30C083EE39C0809142
:1010D000EE0182FD28C0F5CF8091EE0183FF27C08D
:1010E0008091EE0184FD21C087EE2AC08091EE013F
:1010F00083FD1DC0F5CF8091EE0185FD1AC01BC098
:101100008091EE0185FD17C014C08091EE0186FD2F
:1011100014C015C08091EE0186FD11C00EC080EE96
:101120000FC089E30DC082EE0BC080E009C086EEDF
:1011300007C089E205C085E303C08AE201C081E3FC
:1011400090E0089508950C94A20880916F0108958D
:10115000CF93DF9300D01F92CDB7DEB79C01809173
:10116000F401843019F593E099833B832A839093AB
:10117000E9008FEF9091E800815095FD06C095ED54
:101180009A95F1F700008111F5CF8091E80085FF75
:101190000DC040E050E063E070E0CE0101960E9497
:1011A0000E0B8091E8008E778093E8000F900F90EF
:1011B0000F90DF91CF910895CF93DF9300D01F92CE
:1011C000CDB7DEB72091F401243021F522E0298348
:1011D0009B838A8383E08093E9008FEF9091E800FE
:1011E000815095FD06C095ED9A95F1F700008111AB
:1011F000F5CF8091E80085FF0DC040E050E063E04E
:1012000070E0CE0101960E940E0B8091E8008E776F
:101210008093E8000F900F900F90DF91CF91089589
:101220002091F4012430F1F422E02093E9002FEF23
:101230003091E800215035FD06C035ED3A95F1F7C3
:1012400000002111F5CF2091E80025FF0BC040E000
:1012500050E065E070E00E940E0B8091E8008E7710
:101260008093E8000895CF93DF93EC019091F4010F
:10127000943009F046C080910C018823D9F0809108
:101280000D018823B9F09093E9008FEF9091E80069
:10129000815095FD06C095E19A95F1F70000811106
:1012A000F5CF8091E80085FF2CC040E050E060E180
:1012B00070E017C081E08093E9008FEF9091E80023
:1012C000815095FD06C095ED9A95F1F700008111CA
:1012D000F5CF8091E80085FF14C040E050E068E061
:1012E00070E0CE010E940E0B8091E8008E77809313
:1012F000E80080E1FE01AFE5B1E001900D928A9532
:10130000E1F7DF91CF9108958091F301811109C038
:101310000E94A30C0E94000D8091E20084608093E3
:10132000E20008951092F301089508950C94472067
:101330000E94F71A0E944D200E94A60F0C94A30849
:1013400042E061EC81E00E941D0C42E061EC82E031
:101350000E941D0C42E061EC83E00E941D0C42E102
:1013600061EC84E00C941D0C8091F601833009F44B
:1013700055C030F4813071F0823009F48EC0089588
:101380008A3009F47AC08B3009F460C0893009F0E2
:101390009CC020C08091F501813A09F096C08091EF
:1013A000E800877F8093E8008091F9019091FA012D
:1013B000892B21F460E18FE591E003C060E080E0DB
:1013C00090E070E00E94590B8091E8008B77809349
:1013D000E80008958091F501813209F076C080918E
:1013E000F9019091FA01009719F0039709F06DC087
:1013F0008091E800877F8093E8008091E80082FD7B
:1014000005C08091F4018111F8CF5FC08091F10097
:1014100080936F018091E8008B7753C08091F50134
:10142000813A09F052C08091F9019091FA01892B1B
:1014300009F04BC08091E800877F8093E80080919D
:10144000E80080FFFCCF80910C0136C08091F5014F
:101450008132D9F58091F9019091FA01892BA9F592
:101460008091E800877F8093E8000E94520C809171
:10147000F70180930C010C943F148091F5018132A7
:1014800021F58091E800877F8093E8000E94520C4C
:101490008091F8018093700108958091F501813A5F
:1014A000A1F48091E800877F8093E8008091E800B4
:1014B00080FFFCCF809170018093F1008091E80063
:1014C0008E778093E8000C94520C089584B7877F40
:1014D00084BF88E10FB6F89480936000109260009A
:1014E0000FBE80E880936100109261000E94F50FAA
:1014F0000E94A30C0E94000D8091E2008460809302
:10150000E20078940E94860F0E94F70F82E091E03B
:101510000E94A10F0E9435208091F401853069F46A
:101520000E94BF1A8091F2018823B1F30E94E91A48
:10153000882391F30E94F80AEFCF0E94FD0FECCFB1
:10154000292F332723303105C9F064F421303105C8
:1015500081F02230310509F043C08DE690E026EE9F
:1015600031E042C021323105F1F02232310541F142
:1015700037C082E190E023E532E036C09927813020
:10158000910541F08230910541F0892B49F5E2EE59
:10159000F1E005C0EAECF1E002C0E2EBF1E0849199
:1015A00090E09F0121C06430D8F4E62FF0E0EE0F08
:1015B000FF1FEE5DFE4F2081318189E090E014C075
:1015C000643070F470E0FB01EE0FFF1FE65EFE4F2B
:1015D00020813181FB01EA5EFE4F808190E004C0F2
:1015E00080E090E020E030E0FA013183208308952C
:1015F00080E189BD82E189BD09B400FEFDCF809103
:10160000D8008F7D8093D8008091E0008260809325
:10161000E0008091E00081FDFCCF0895CF92DF9241
:10162000EF92FF920F931F93CF93DF93EC018B0107
:101630006A010E94710C811133C0C114D10439F0C8
:10164000F60180819181081B190BC80FD91FE12C6D
:10165000F12C0115110519F18091E80085FD16C0E6
:101660008091E8008E778093E800C114D10449F09E
:10167000F60180819181E80EF91EF182E08285E019
:101680000FC00E94710C882321F30AC089918093B6
:10169000F10001501109FFEFEF1AFF0ADACF80E0E5
:1016A000DF91CF911F910F91FF90EF90DF90CF903E
:1016B00008952091FB013091FC012617370748F06F
:1016C0006115710539F42091E8002E772093E80028
:1016D00001C0B90140E061157105A9F12091F40143
:1016E000222309F443C0253009F442C02091E800C8
:1016F00023FD40C02091E80022FD32C02091E80087
:1017000020FFE9CF4091F3002091F20030E0342B2C
:10171000FC01CF016115710559F02830310540F405
:1017200081918093F100615071092F5F3F4FF1CF9C
:1017300041E02830310509F040E02091E8002E77A3
:101740002093E800C8CF4111C9CF0AC08091F401AD
:10175000882361F0853061F08091E80083FD0AC044
:101760008091E80082FFF2CF80E0089582E0089542
:1017700083E0089581E008952091FB013091FC0100
:101780002617370748F06115710539F42091E800F4
:101790002E772093E80001C0B901FC0120E061151B
:1017A000710591F18091F401882309F440C08530DE
:1017B00009F43FC08091E80083FD3DC08091E800BE
:1017C00082FD2FC08091E80080FFE9CF2091F300D7
:1017D0008091F20090E0922B6115710559F08830EC
:1017E000910540F424912093F100319661507109E4
:1017F0000196F2CF21E0089709F020E08091E800FF
:101800008E778093E800CBCF2111CCCF0AC0809196
:10181000F401882361F0853061F08091E80083FD58
:101820000AC08091E80082FFF2CF80E0089582E054
:10183000089583E0089581E00895982F973058F532
:101840009093E900981739F07091EC002091ED0029
:101850005091F00003C0242F762F50E021FF19C0D3
:101860003091EB003E7F3093EB003091ED003D7FF7
:101870003093ED003091EB0031603093EB007093CA
:10188000EC002093ED005093F0002091EE0027FF34
:1018900007C09F5FD3CF8F708093E90081E00895E8
:1018A00080E008958091F50187FF11C08091E800E4
:1018B00082FD05C08091F4018111F8CF11C08091A3
:1018C000E8008B770BC08091F401882349F0809168
:1018D000E80080FFF8CF8091E8008E778093E800E1
:1018E00008952091E4003091E50095E64091EC00E8
:1018F000842F817040FF22C08091E80080FD1CC0D1
:101900008091F401882391F0853091F08091EB0073
:1019100085FD10C04091E4005091E5004217530747
:1019200029F39A01915011F784E0089582E0089517
:1019300083E0089581E0089580E008954091E800F3
:1019400042FFDECF08950E94110D0E94190DE0EEB6
:10195000F0E0808181608083E8EDF0E080818F7726
:10196000808319BCA7EDB0E08C918E7F8C93808131
:101970008F7E80831092F30108950F931F93CF936E
:10198000DF930E94110D0E94190DC8EDD0E08881EF
:101990008F77888388818068888388818F7D88831A
:1019A00019BC1092F4011092F0011092F201109201
:1019B000F10100EE10E0F80180818B7F8083888147
:1019C0008160888342E060E080E00E941D0CE1EECF
:1019D000F0E080818E7F8083E2EEF0E080818160A4
:1019E0008083808188608083F80180818E7F8083FE
:1019F000888180618883DF91CF911F910F91089535
:101A0000E8EDF0E080818F7E8083E7EDF0E080817B
:101A10008160808384E082BF81E08093F3010C9435
:101A2000BD0CE8EDF0E080818E7F80831092E200B3
:101A300008951092DA001092E10008951F920F921B
:101A40000FB60F9211242F933F934F935F936F9391
:101A50007F938F939F93AF93BF93EF93FF93809167
:101A6000E10082FF0BC08091E20082FF07C08091FD
:101A7000E1008B7F8093E1000E94850F8091DA0066
:101A800080FF1FC08091D80080FF1BC08091DA00CA
:101A90008E7F8093DA008091D90080FF0DC080E1B5
:101AA00089BD82E189BD09B400FEFDCF81E080934C
:101AB000F4010E94840905C019BC1092F4010E942F
:101AC00092098091E10080FF19C08091E20080FFBF
:101AD00015C08091E2008E7F8093E2008091E20049
:101AE00080618093E2008091D80080628093D8006A
:101AF00019BC85E08093F4010E9496098091E10071
:101B000084FF30C08091E20084FF2CC080E189BD59
:101B100082E189BD09B400FEFDCF8091D8008F7DA0
:101B20008093D8008091E1008F7E8093E1008091C6
:101B3000E2008F7E8093E2008091E20081608093DA
:101B4000E2008091F001882311F084E007C08091C9
:101B5000E30087FD02C081E001C083E08093F401CF
:101B60000E9498098091E10083FF29C08091E200E2
:101B700083FF25C08091E100877F8093E10082E0B0
:101B80008093F4011092F0018091E1008E7F8093A8
:101B9000E1008091E2008E7F8093E2008091E2007C
:101BA00080618093E20042E060E080E00E941D0CD2
:101BB0008091F00088608093F0000E949509FF9169
:101BC000EF91BF91AF919F918F917F916F915F91B5
:101BD0004F913F912F910F900FBE0F901F9018952E
:101BE0001F920F920FB60F9211242F933F934F9392
:101BF0005F936F937F938F939F93AF93BF93CF9395
:101C0000DF93EF93FF93C091E900CF708091EC00D8
:101C1000D82FD17080FDD0E81092E9008091F000BB
:101C2000877F8093F00078940E94340E1092E90030
:101C30008091F00088608093F000CD2BCF70C0932E
:101C4000E900FF91EF91DF91CF91BF91AF919F910B
:101C50008F917F916F915F914F913F912F910F9055
:101C60000FBE0F901F9018951F93CF93DF93CDB7A2
:101C7000DEB7AA970FB6F894DEBF0FBECDBFE5EF73
:101C8000F1E088E08E0F9091F10091938E13FBCFDD
:101C90000E94B4098091E80083FF1FC18091F50183
:101CA0009091F601492F50E04A30510508F015C1D6
:101CB000FA01EA5AFF4F0C94CF21803881F0823824
:101CC00009F00BC18091F9018F708093E900809138
:101CD000EB0085FB882780F91092E90006C080910F
:101CE000F1019091F201911182609091E800977F4B
:101CF0009093E8008093F1001092F100C8C0282F63
:101D00002D7F09F0EAC0882319F0823061F0E5C028
:101D10008091F701813009F0E0C0933009F080E054
:101D20008093F2012BC08091F701811127C080912F
:101D3000F9018F7009F4D1C08093E9002091EB0084
:101D400020FF1CC0933021F48091EB00806214C00E
:101D50009091EB0090619093EB0021E030E0A901BD
:101D600002C0440F551F8A95E2F74093EA00109293
:101D7000EA008091EB0088608093EB001092E9000C
:101D80008091E800877F86C08111A7C01091F7017C
:101D90001F778091E3008078812B8093E30080910E
:101DA000E800877F8093E8000E94520C8091E80051
:101DB00080FFFCCF8091E30080688093E3001111E5
:101DC00002C082E001C083E08093F40186C08058A5
:101DD000823008F082C08091F7019091F8018C3D2B
:101DE00053E0950779F583E08A838AE289834FB7C8
:101DF000F894DE01139620E03EE051E2E32FF0E09C
:101E000050935700E49120FF03C0E295EF703F5FCD
:101E1000EF708E2F90E0EA3010F0C79601C0C096A8
:101E20008D939D932F5F243149F74FBF8091E80038
:101E3000877F8093E8006AE270E0CE0101960E94FD
:101E4000590B14C0AE014F5F5F4F6091F9010E94C2
:101E5000A00ABC01009709F440C09091E800977F68
:101E60009093E80089819A810E94BC0B8091E800E0
:101E70008B778093E80031C0803879F58091E80055
:101E8000877F8093E8008091F0018093F10080913A
:101E9000E8008E778093E8000E94520C1EC08111EA
:101EA0001CC09091F7019230C0F48091E800877FC8
:101EB0008093E8009093F0010E94520C8091F00111
:101EC000811106C08091E30087FD02C081E001C05E
:101ED00084E08093F4010E94A0098091E80083FFD0
:101EE0000AC08091E800877F8093E8008091EB0032
:101EF00080628093EB00AA960FB6F894DEBF0FBE07
:101F0000CDBFDF91CF911F9108950895CF93809118
:101F1000F4018823A1F0C091E900CF709091EC000A
:101F2000892F817090FD80E8C82B1092E900809184
:101F3000E80083FD0E94340ECF70C093E900CF917A
:101F4000089590937601809375010895E09175014D
:101F5000F0917601309721F00190F081E02D099405
:101F600080E00895E0917501F0917601309721F0BD
:101F70000280F381E02D09940895E0917501F091BC
:101F80007601309721F00480F581E02D09940895C1
:101F900020917301309174018217930771F090932F
:101FA000740180937301E0917501F091760130978F
:101FB00021F00680F781E02D0994089520917101A8
:101FC000309172018217930771F0909372018093A0
:101FD0007101E0917501F0917601309721F0008454
:101FE000F185E02D0994089508950C94F40F0E9452
:101FF000FD1A0E9491020C94831B9F92AF92BF9294
:10200000CF92DF92EF92FF920F931F93CF93DF93C4
:1020100000D000D000D0CDB7DEB70E94B8020DE0EE
:1020200010E0AA24A394B12C902E802F0E94A60326
:10203000980128583E4F6901F901F080F826A1F473
:102040000150110988F78FEF89838A831B820E94D0
:10205000061B8160782F9D838C8349815A816B8117
:102060008D810E9494102FC09091DB0191FF04C0DC
:102070008E830E94AC038E8125E030E0A501022E04
:1020800001C0440F0A94EAF7E42E4F21C1F02983DE
:102090009A828E2191E009F490E09B830E94061BB6
:1020A0008160782F9D838C8349815A816B818D81DA
:1020B0000E949410F6018081E826E08204C021503D
:1020C0003109E0F6BDCF0E94511D109177010E94A9
:1020D000A60F1817B9F00E94A60F809377012696D5
:1020E0000FB6F894DEBF0FBECDBFDF91CF911F9129
:1020F0000F91FF90EF90DF90CF90BF90AF909F90A7
:102100000C94A30826960FB6F894DEBF0FBECDBF81
:10211000DF91CF911F910F91FF90EF90DF90CF90C3
:10212000BF90AF909F900895CF93DF93CDB7DEB768
:102130002B970FB6F894DEBF0FBECDBF4F835887E5
:1021400069877A878B87DE01119686E0FD011192FF
:102150008A95E9F785E0FE01379601900D928A9500
:10216000E1F749815A816B817C818D819E810E943A
:10217000DD162B960FB6F894DEBF0FBECDBFDF91F4
:10218000CF910895CF93882309F4C2C0C82F823815
:1021900059F40E94A60F81FDBBC089E30E94B719C4
:1021A0000E94841A89E30CC0833879F40E94A60F38
:1021B00080FDAEC083E50E94B7190E94841A83E5B2
:1021C0000E94F919CF910C94841A843859F40E9412
:1021D000A60F82FD9DC087E40E94B7190E94841A51
:1021E00087E4EECF8CEF8C0F813A48F48C2F0E945D
:1021F0009B1F81118DC08C2F0E94B719E3CF80E205
:102200008C0F883048F4C77081E001C0880FCA95F0
:10221000EAF70E943D1AD6CF8BE58C0F833078F415
:10222000C53A29F0C63A31F083E890E005C081E86C
:1022300090E002C082E890E0CF910C94C80F88E54E
:102240008C0F833108F064C0C83A39F1C93A41F1C2
:10225000CA3A49F1CB3A51F1CC3A59F1CD3A61F150
:10226000C03B69F1CE3A71F1CF3A79F1C13B81F1CE
:10227000C23B89F1C33B91F1C43B99F1C53BA1F14C
:10228000C63BA9F1C73BB1F1C83BB9F1C93BC1F1AC
:10229000CA3BC9F180E090E038C082EE90E035C0E2
:1022A00089EE90E032C08AEE90E02FC085EB90E09E
:1022B0002CC086EB90E029C087EB90E026C08CEC28
:1022C00090E023C08DEC90E020C083E891E01DC039
:1022D0008AE891E01AC082E991E017C084E991E0B0
:1022E00014C081E292E011C083E292E00EC084E269
:1022F00092E00BC085E292E008C086E292E005C061
:1023000087E292E002C08AE292E0CF910C94DE0F65
:10231000CF910895882309F44BC0823859F40E9464
:10232000A60F81FF45C089E30E94B7190E94841A55
:1023300089E30CC0833871F40E94A60F80FF38C077
:1023400083E50E94B7190E94841A83E50E94F91957
:102350000C94841A843859F40E94A60F82FF28C076
:1023600087E40E94B7190E94841A87E4EFCF9CEF9C
:10237000980F913A58F390E2980F983050F4877084
:1023800091E001C0990F8A95EAF7892F0E94431ABC
:10239000DFCF9BE5980F933020F480E090E00C9421
:1023A000C80F885A833120F480E090E00C94DE0F4F
:1023B0000895882321F00E943D1A0C94841A0895F0
:1023C000882321F00E94431A0C94841A08957F9266
:1023D0008F929F92AF92BF92CF92DF92EF92FF9235
:1023E0000F931F93CF93DF931F92CDB7DEB77C017E
:1023F000C62E772EFC01058102950F7012811111F6
:102400000E945A1A0E94B019882379F0112369F0AA
:1024100080E28C0D883048F082E00E9499190E9479
:10242000B01991E0D82ED92601C0D12CE72DE29524
:10243000EF70F0E0E05AFF4F0C94CF21872D807FA2
:10244000072D0F70882311F00295007F112389F06A
:10245000002309F490C180E28C0D883020F4802F95
:102460000E943D1A03C0802F0E944D1A0E94841AB8
:1024700082C18C2D0E948A11002309F495C180E24B
:102480008C0D883020F4802F0E94431A03C0802FC7
:102490000E94531A0E94841A87C1972D907F872D1E
:1024A0008F70903211F08295807FCC2021F0F1E086
:1024B000CF16B1F01EC0112349F0002309F414C156
:1024C000013009F011C10E946D1A6EC1002319F08C
:1024D000013009F469C189830E94701A89810AC197
:1024E000112321F0023008F05FC1FEC001115CC170
:1024F00001C1112321F0002309F4F6C03CC10023DF
:1025000009F4F8C03EC1872D86958695837090E0CA
:10251000009719F0019761F047C1112321F08C2D2C
:10252000972D937002C080E090E00E94C80F3CC1DC
:10253000112321F08C2D972D937002C080E090E044
:102540000E94DE0F31C18C2D112319F00E94591CFD
:1025500002C00E94C11C0E94461D26C1872D8370A7
:1025600009F052C0111120C18C2D8295869587707B
:10257000880F880F9C2D9F70892E912CA12CB12C37
:10258000082E04C0880C991CAA1CBB1C0A94D2F704
:10259000C4FE14C00FE010E020E030E0B901A80153
:1025A00004C0440F551F661F771F8A95D2F7CB01D1
:1025B000BA01609570958095909503C060E070E0D9
:1025C000CB01272D26952695237030E0223031054A
:1025D00069F02330310589F0682979298A299B29F6
:1025E0002130310571F00E942518DEC06829792953
:1025F0008A299B290E944118D7C00E942518C5012D
:10260000B4010E940918D0C0112319F0872D8170E0
:1026100001C08695882309F4C7C08C2D82958695C4
:102620008770880F880F9C2D9F70892E912CA12C6C
:10263000B12C082E04C0880C991CAA1CBB1C0A943F
:10264000D2F7C4FE14C00FE010E020E030E0B90182
:10265000A80104C0440F551F661F771F8A95D2F743
:10266000CB01BA01609570958095909503C060E0AC
:1026700070E0CB01272D269526952370422F50E040
:102680004230510569F04330510589F068297929B4
:102690008A299B294130510571F00E94FF1884C09E
:1026A000682979298A299B290E941B197DC00E94CB
:1026B000FF18C501B4010E94E31876C08C2D90E08C
:1026C000FC01E05EF109E531F10508F050C0E05988
:1026D000FF4F0C94CF210C2D0F70872D8F7111237C
:1026E00031F00E947C18802F0E94D9115DC00E9499
:1026F0009D18802F0E94E01157C0112339F001115D
:1027000053C0872D8F710E94C2184EC0023008F04E
:102710004BC0F7CF112339F0872D8F710E947C18A1
:1027200043C01123C9F3872D8F710E949D183CC0AF
:10273000112329F0872D8F710E94671835C00E94E0
:102740005D1832C0112351F0172D1F71812F0E9487
:102750007C1863E0812F0E94901926C081E00E94BE
:102760009919023008F182E00E9499191DC01123C5
:1027700031F0002389F28C2D0E94C21015C0002375
:1027800091F28C2D0E948A110FC0472D4F706C2D35
:10279000C7010E9482040E94811706C0472D4F7016
:1027A0006C2DC7010E941208DD20F9F00E948C19DF
:1027B00080FD1BC0F70112820E9486190E947C18BE
:1027C000C7010E9404140E9486190F90DF91CF91D7
:1027D0001F910F91FF90EF90DF90CF90BF90AF903F
:1027E0009F908F907F900C949D180F90DF91CF91C8
:1027F0001F910F91FF90EF90DF90CF90BF90AF901F
:102800009F908F907F9008950F931F93CF93DF93A6
:10281000EC01888199812B813C81232BB9F09F3F6A
:1028200011F48F3F99F0CE010E94A304882371F028
:10283000688179818A810E9482198C010E943719EE
:102840000E94FE17B801CE010E94E711DF91CF91DF
:102850001F910F9108950E945A1A0E946A1A0E94AD
:102860002F1A0E94841A0E94F71D0E94461D80E0C4
:1028700090E00E94C80F80E090E00C94DE0F0E9470
:102880004A1A0C942B140E947719292F22952F7025
:1028900030E02C3031054CF42A3031056CF42250F4
:1028A000310922303105A8F407C02C30310569F018
:1028B0002F30310551F00DC0803F69F018F4803E93
:1028C00040F409C0843F29F406C093FB882780F9AF
:1028D000089580E0089581E00895CF93DF9300D0BC
:1028E00000D01F92CDB7DEB70F900F900F900F90D2
:1028F0000F90DF91CF910895CF93DF9300D000D058
:1029000000D0CDB7DEB726960FB6F894DEBF0FBE67
:10291000CDBFDF91CF9108951F93CF93DF93C091E7
:10292000860116E080918701C81799F0D0E01C9FBE
:10293000F0011D9FF00D1124E857FE4F4081518199
:1029400062817381848195810E947C142196C77075
:10295000E9CFDF91CF911F9108954091B801509137
:10296000B9016091BA017091BB018091BC01909155
:10297000BD010C947C148091BD0182958F7009F08B
:1029800054C08091BA01882309F44FC08091860118
:10299000A09187016091B8017091B9014091BB018C
:1029A0005091BC01B6E08A1709F43FC090E0411590
:1029B0005105C1F17F3F11F46F3FA1F1B89FF001C4
:1029C000B99FF00D1124E857FE4F218172132AC0E0
:1029D0002081621327C02281211124C023813481E8
:1029E0002417350710F421503109241B350B283CDE
:1029F0003105C0F42091BD012F7020612093BD01ED
:102A000026E0289FF001299FF00D1124E357FE4F87
:102A100080818F708061808388EB91E00E94041434
:102A20000C948C1401968770BECF0895CF92DF92DC
:102A3000EF92FF920F931F93CF93DF93CDB7DEB743
:102A400062970FB6F894DEBF0FBECDBF8C0185E054
:102A5000F801DE011D9601900D928A95E1F7D801EB
:102A60004C9111965C91119712966C911297139656
:102A7000CD90DC9014973091B8017091B90180919C
:102A8000BB019091BC01009709F46BC17F3F19F421
:102A90003F3F09F466C1E090BA01EE2009F4C0C0DE
:102AA0002091BD01C816D90628F0F601E81BF90BE4
:102AB000CF0104C0809590958C0D9D1DFF24F3944B
:102AC000883C910578F0F12C207F09F0C6C07C2D60
:102AD000D98AC88A89890E946D1488EB91E00E9486
:102AE0000414B1C0822F807F09F046C0751314C052
:102AF000341312C0611110C02F7020612093BD01EA
:102B00000E94AD1488EB91E00E9404148091BD01F5
:102B1000D80115968C932EC0CD2819F15F3F11F482
:102B20004F3FF9F0F62E61111CC080918601209173
:102B3000870136E0821709F45AC090E0389FF0010F
:102B4000399FF00D1124E857FE4F7181571306C0CD
:102B50007081471303C07281711103C001968770A1
:102B6000E9CFF62E662309F418C18091BD0181607A
:102B70008093BD01F12C11C1751308C0341306C038
:102B8000611104C08091BD01D801C3C04D875E872B
:102B90008D859E856A8B0E9443146A898823E1F1A2
:102BA0006623D1F12091BD01822F82958F7090E034
:102BB000029774F08091B8019091B90198878F8342
:102BC0001986DB86CA862C87CE0107960E940414DC
:102BD00086E0F801A8EBB1E001900D928A95E1F74B
:102BE0000E94BB140E94AD14FF24F394D6C04D87FD
:102BF0005E878D859E850E947719292F22952F70DB
:102C000030E0223031050CF0BCC09F7009F0B6C036
:102C1000805E883008F4C1C0C8010E940414E4CF6B
:102C2000C816D90608F453C0F601E81BF90BCF010A
:102C3000883C910508F450C0F12C7C2DD98AC88AB3
:102C400089890E946D14E8EBF1E086E0DF011D92B6
:102C50008A95E9F70E94AD14A0C0751314C034130F
:102C600012C0611110C08091BD01F8018583C801B7
:102C70000E94041486E0E8EBF1E0DF011D928A95E2
:102C8000E9F7FE2C8AC04D875E878D859E856A8B0D
:102C90000E9443146A89882309F4BECF662309F48D
:102CA000BBCF2091BD01822F82958F7090E002975B
:102CB0000CF48ECF8091B8019091B9019A838983E9
:102CC0001B82DD82CC822E83CE0101967FCF809540
:102CD00090958C0D9D1DACCFF62E662309F49CCFEC
:102CE00075132EC034132CC02091BD0120FD1FC0D0
:102CF000822F82958F70D9F0D80115962C93159755
:102D00008F3049F08F5F982F9295907F822F8F7030
:102D1000892B15968C93C8010E94041486E0F80153
:102D2000A8EBB1E001900D928A95E1F793CF86E090
:102D3000F801A8EBB1E001900D928A95E1F72DC062
:102D40004D875E878D859E850E944314811140CFFB
:102D50008091BD0181608093BD01C8010E9404146F
:102D60001CC0662309F458CF4D875E878D859E85EC
:102D70000E944314882309F44FCF2ACF811148CFF2
:102D80000CC0243031050CF047CF9F7009F440CFC0
:102D9000F8019581907F09F03BCF8F2D62960FB699
:102DA000F894DEBF0FBECDBFDF91CF911F910F9181
:102DB000FF90EF90DF90CF9008951F93CF93DF9314
:102DC000CDB7DEB72C970FB6F894DEBF0FBECDBFE0
:102DD0004F83588769877A878B879C87CE010796B0
:102DE0000E941615882369F08F8198852A853B8576
:102DF000232BF1F19F3F09F063C08F3F09F060C0C2
:102E000037C086E0FE013796DE01119601900D92E3
:102E10008A95E1F76F817885EA85FB85309741F1E6
:102E20007F3F11F46F3F21F12091870130E0C9010C
:102E30000196877099274091860150E08417950785
:102E400009F447C069837A83FD83EC8396E0929FFF
:102E5000D001939FB00D1124A857BE4FFE013196AB
:102E600001900D929A95E1F7809387010E948C144E
:102E700016E080918601909187018917C1F1189F12
:102E8000C001112488579E4F0E941615882379F19E
:102E9000E09186011E9FF0011124E857FE4F40810A
:102EA000518162817381848195810E947C1480911B
:102EB000860190E001968770992780938601D9CF8B
:102EC0004F81588569857A858B859C850E947C1405
:102ED000CFCF0E943F141092870110928601E8EB39
:102EE000F1E086E0DF011D928A95E9F7C1CF2C96CB
:102EF0000FB6F894DEBF0FBECDBFDF91CF911F910B
:102F00000895EF92FF920F931F93CF93DF938C015D
:102F1000009709F46CC0F12CEE24E394E8012196AB
:102F2000F8018491843740F4843008F051C0813036
:102F300081F0823019F15BC0853709F444C0A8F1F3
:102F40009CE7980F903708F052C08F770E948A1143
:102F500041C00E5F1F4FFE01C49180E28C0F88308C
:102F600048F4C7708E2D01C0880FCA95EAF70E94F9
:102F70005D1A14C08C2F0E94C2102DC00E5F1F4F0F
:102F8000FE01C49180E28C0F883058F4C7708E2DFA
:102F900001C0880FCA95EAF70E94631A0E94841A3A
:102FA0001AC08C2F0E948A1116C00E5F1F4FFE019F
:102FB000C491CC2381F08FE99FE00197F1F700C025
:102FC0000000C150F6CF0E5F1F4FFE01F49003C00A
:102FD0000E94C2108E018F2D882309F49FCFEFE944
:102FE000FFE03197F1F700C000008150F5CFDF918D
:102FF000CF911F910F91FF90EF90089508956093E6
:10300000C2017093C3018093C4019093C5010C94D5
:103010002B140F931F930091C2011091C3012091B3
:10302000C4013091C501DC01CB01802B912BA22B77
:10303000B32B8093C2019093C301A093C401B093BA
:10304000C5011F910F910C942B140F931F930091A6
:10305000C2011091C3012091C4013091C501DC016E
:10306000CB0180239123A223B3238093C2019093A9
:10307000C301A093C401B093C5011F910F910C949B
:103080002B140F931F930091C2011091C301209143
:10309000C4013091C501DC01CB0180279127A22713
:1030A000B3278093C2019093C301A093C401B0934E
:1030B000C5011F910F910C942B141092BE01109218
:1030C000BF011092C0011092C1010C942B1441E079
:1030D00050E060E070E004C0440F551F661F771F8A
:1030E0008A95D2F74093BE015093BF016093C0010F
:1030F0007093C1010C942B1441E050E060E070E04B
:1031000004C0440F551F661F771F8A95D2F7809120
:10311000BE019091BF01A091C001B091C101482BA7
:10312000592B6A2B7B2B4093BE015093BF016093B8
:10313000C0017093C1010C942B1441E050E060E099
:1031400070E004C0440F551F661F771F8A95D2F7A1
:1031500040955095609570958091BE019091BF010A
:10316000A091C001B091C101482359236A237B2358
:103170004093BE015093BF016093C0017093C101A1
:103180000C942B1441E050E060E070E004C0440F68
:10319000551F661F771F8A95D2F78091BE019091C7
:1031A000BF01A091C001B091C101482759276A27EA
:1031B0007B274093BE015093BF016093C001709381
:1031C000C1010C942B140F931F930091BE01109119
:1031D000BF012091C0013091C101DC01CB01802BE6
:1031E000912BA22BB32B8093BE019093BF01A09390
:1031F000C001B093C1011F910F910C942B140F9338
:103200001F930091BE011091BF012091C001309128
:10321000C101DC01CB0180239123A223B32380933E
:10322000BE019093BF01A093C001B093C1011F9153
:103230000F910C942B140F931F930091BE011091CA
:10324000BF012091C0013091C101DC01CB01802779
:103250009127A227B3278093BE019093BF01A0932B
:10326000C001B093C1011F910F910C942B140895CC
:10327000CF92DF92EF92FF920F931F93CF93DF9342
:103280008C01C090C201D090C301E090C401F090C5
:10329000C5018091BE019091BF01A091C001B09184
:1032A000C101C82AD92AEA2AFB2ACFE1D0E0D701F6
:1032B000C6010C2E04C0B695A795979587950A94DC
:1032C000D2F780FF06C0B8018C2F0E9491060197AB
:1032D00021F4219760F780E001C08C2FDF91CF911E
:1032E0001F910F91FF90EF90DF90CF900895CF93B3
:1032F000DF93EC010E943819BE010E949106DF9114
:10330000CF910895CB010E94771908958091C6014D
:1033100085958595859508958091C6018770089556
:1033200098E0899F90011124262B2093C6010C94CC
:103330007C182091C601809582238093C601982F26
:10334000977069F430E0482F552747FD50952417B2
:10335000350729F08595859585950C949D180895D8
:103360009091C601977081E009F480E008959091F2
:103370000C01992321F090910D01911109C0209128
:103380000E0130910F01F90132969FEF40E01FC00E
:10339000982F9695969596959F3050F5E0910E0151
:1033A000F0910F01E90FF11D877021E030E0A901D4
:1033B00002C0440F551F8A95E2F7CA019181892BFB
:1033C000818308959F3F39F04F5F4E3041F0519116
:1033D0005813F8CF0DC05111F7CF942FF5CF9F3F61
:1033E00039F0F901E90FF11D97FDFA9582830895EF
:1033F000089590910C01992321F090910D01911164
:1034000009C020910E0130910F01F9013296205F21
:103410003F4F1FC0982F9695969596959F30F0F444
:10342000E0910E01F0910F01E90FF11D877021E08D
:1034300030E0A90102C0440F551F8A95E2F7CA0186
:10344000809591818923818308953196E217F3074E
:1034500029F090819813F9CF1082F7CF089581E079
:1034600090E0E0910E01F0910F01E80FF91F10823A
:10347000019680319105A9F708959091DA01892B81
:103480008093DA01089580959091DA0189238093E1
:10349000DA0108951092DA0108959091D901892BEB
:1034A0008093D901089580959091D90189238093C3
:1034B000D90108951092D90108959091D801892BCE
:1034C0008093D801089580959091D80189238093A5
:1034D000D80108951092D80108958093C7010895E6
:1034E0001092C701089580910E0190910F01FC0187
:1034F00031969C01205F3F4F80E0919191118F5F49
:10350000E217F307D1F70895E0910E01F0910F0152
:103510008091DA018083E0910E01F0910F0190819A
:103520008091D901892B8083E0910E01F0910F01E8
:1035300090818091D801892B80838091C701882355
:1035400061F0E0910E01F0910F019081892B808351
:103550000E94731A81111092C70180910E019091FF
:103560000F010C94B20F20E0009739F0AC014150EC
:103570005109842395232F5FF7CF822F08958091DF
:10358000F401843021F11092DC0120E488E190E024
:103590000FB6F894A895809360000FBE209360004A
:1035A00080E00E94A30883B7817F846083BF83B7D4
:1035B000816083BF7894889583B78E7F83BF88E1CD
:1035C0000FB6F89480936000109260000FBE0895CB
:1035D00008950E94A5020E94B8020E94E81A0E9463
:1035E000AD0391E0811101C090E0892F08950E9400
:1035F0003F140E94A60F0C94A30882E084BD93E0C0
:1036000095BD9AEF97BD80936E0008952FB7F894FB
:103610008091DD019091DE01A091DF01B091E00188
:103620002FBF0895CF92DF92EF92FF920F931F93D7
:103630002FB7F8944091DD015091DE016091DF01D8
:103640007091E0012FBF6A017B01EE24FF248C0101
:1036500020E030E0C016D106E206F30610F4415037
:1036600051099A01281B390BC9011F910F91FF9035
:10367000EF90DF90CF9008951F920F920FB60F92A8
:1036800011248F939F93AF93BF938091DD0190910D
:10369000DE01A091DF01B091E0010196A11DB11DF5
:1036A0008093DD019093DE01A093DF01B093E001F0
:1036B000BF91AF919F918F910F900FBE0F901F9070
:1036C00018950E94A30CF8942FEF87EA91E62150F9
:1036D00080409040E1F700C0000087E090EBDC0103
:1036E0008093FD019093FE01A093FF01B09300022F
:1036F0009CE088E10FB6F894A895809360000FBE17
:1037000090936000FFCF0E94BB1B811102C00E94FA
:10371000A11B0E94C61B8093DB010E94CE1B90E080
:103720009093EF018093EE0187FB882780F98093C7
:103730000D010E94CA1B682F70E080E090E00C949D
:10374000FF176DEE7EEF80E090E00E94092260E0BE
:1037500082E090E00E94F72160E083E090E00E9428
:10376000F72160E084E090E00E94F72160E085E0CE
:1037700090E00C94F72180E090E00E94F12121E09C
:103780008D3E9E4F09F020E0822F089582E090E068
:103790000C94E92183E090E00C94E92184E090E02E
:1037A0000C94E921682F84E090E00C94F72180913B
:1037B000E30180FF0BC06091130185E0689FB001B9
:1037C000112475956795759567952BC081FF09C084
:1037D0006091130185E0689FB0011124759567958C
:1037E00020C082FF07C06091130185E0689FB0018F
:1037F000112417C09091E4019923D1F06091120136
:10380000961788F72091130185E0289F90011124D5
:10381000929FA001939F500D112470E0CA010E9455
:10382000BB216038710540F46115710539F002C0A3
:1038300065E070E0862F08958FE7089581E0089590
:103840008091E30180FF08C06091110170E07595DF
:1038500067957595679521C081FF06C0609111013C
:1038600070E07595679519C082FF04C060911101E1
:1038700070E010C09091E4019923C1F060911001B3
:103880009617A0F780911101899FC001112470E063
:103890000E94BB216038710528F46115710521F083
:1038A000862F08958FE7089581E0089561E070E024
:1038B000F4CF803F21F40E94D71B819504C0813F43
:1038C00029F40E94D71B8093E7010895823F21F4D9
:1038D0000E94D71B819504C0833F29F40E94D71B07
:1038E0008093E6010895893F19F40E94201C05C0C9
:1038F0008A3F31F40E94201C81958093E80108954D
:103900008B3F21F40E94201C819504C08C3F29F438
:103910000E94201C8093E9010895843F21F4809146
:10392000E501816017C0853F21F48091E501826047
:1039300011C0863F21F48091E50184600BC0873F70
:1039400021F48091E501886005C0883F31F48091C1
:10395000E50180618093E50108958D3F21F4809118
:10396000E30181600BC08E3F21F48091E30182600E
:1039700005C08F3F29F48091E30184608093E301C7
:103980000895803F39F48091E70187FF6CC0109261
:10399000E70169C0813F29F48091E7011816BCF363
:1039A00062C09091E601823F29F497FF5CC01092BB
:1039B000E60159C0833F19F41916CCF354C0893F6E
:1039C00041F48091E80118160CF04DC01092E80106
:1039D0004AC08A3F29F48091E80187FF44C0F6CFAE
:1039E0008B3F39F48091E90187FF3DC01092E901D6
:1039F0003AC08C3F29F48091E9011816BCF333C01A
:103A0000843F21F48091E5018E7F17C0853F21F42A
:103A10008091E5018D7F11C0863F21F48091E50101
:103A20008B7F0BC0873F21F48091E501877F05C024
:103A3000883F31F48091E5018F7E8093E50113C0CA
:103A40008D3F21F48091E3018E7F0BC08E3F21F4E6
:103A50008091E3018D7F05C08F3F29F48091E301C0
:103A60008B7F8093E3018091E60181110EC08091EC
:103A7000E70181110AC08091E801811106C080919F
:103A8000E901811102C01092E401089585EE91E0F0
:103A90000E94BD0F0E94061B9093E2018093E101FA
:103AA00008951F93CF93DF938091E1019091E201FC
:103AB0000E94121BAC019091E401992321F0209106
:103AC000140130E006C0209115018AE0289F900182
:103AD00011244217530708F486C08091E601C09173
:103AE000E701D091E8011091E901811107C0C111EE
:103AF00076C0D11174C0111172C075C09F3F19F00A
:103B00009F5F9093E401181624F40E94D71B8093C2
:103B1000E6018091E60187FF05C00E94D71B8195D1
:103B20008093E6011C1624F40E94D71B8093E701C2
:103B30008091E70187FF05C00E94D71B8195809384
:103B4000E7016091E601662339F1C091E701CC23DA
:103B500019F1772767FD7095872F972F0E94CC204A
:103B600023E333E343E35FE30E9430210E94992083
:103B70006093E6016C2F772767FD7095872F972F4D
:103B80000E94CC2023E333E343E35FE30E94302130
:103B90000E9499206093E7011D1624F40E94201CC6
:103BA0008093E8018091E80187FF05C00E94201CF6
:103BB00081958093E801111624F40E94201C8093C3
:103BC000E9018091E90187FF05C00E94201C8195D1
:103BD0008093E901DF91CF911F910C94461D9F3F87
:103BE00009F08ECF96CFDF91CF911F910895E5EE2A
:103BF000F1E085E0DF011D928A95E9F71092E4017A
:103C00001092E3010895833081F128F4813059F056
:103C10008230D1F00895853009F449C0B8F186307A
:103C200009F456C0089580911501262F30E0280F21
:103C3000311D2F3F310524F4680F6093150108955D
:103C40008FEF80931501089580911401262F30E0A5
:103C5000280F311D2F3F310524F4680F60931401A4
:103C600008958FEF80931401089580911301262FFA
:103C700030E0280F311D2F3F310524F4680F609389
:103C8000130108958FEF809313010895809112011D
:103C9000262F30E0280F311D2F3F310524F4680F07
:103CA0006093120108958FEF80931201089580911F
:103CB0001101262F30E0280F311D2F3F310524F44C
:103CC000680F6093110108958FEF8093110108959B
:103CD00080911001262F30E0280F311D2F3F310534
:103CE00024F4680F6093100108958FEF8093100102
:103CF0000895833011F128F4813049F0823091F039
:103D00000895853081F120F18630C1F108958091C8
:103D10001501681720F4861B8093150108951092F1
:103D20001501089580911401681720F4861B809373
:103D300014010895109214010895809113016817D9
:103D400020F4861B809313010895109213010895A7
:103D500080911201681720F4861B80931201089548
:103D600010921201089580911101681720F4861BAA
:103D7000809311010895109211010895809110010E
:103D8000681720F4861B809310010895109210018B
:103D900008950F931F938D3109F471C008F045C049
:103DA000803109F485C008F5873009F46FC068F4E4
:103DB000863009F0ADC08091DB01817F8E7F8093DA
:103DC000DB0181E08093EB01A4C08B3009F49EC03D
:103DD0008E3009F09DC08091DB0182FB222720F903
:103DE00091E0922790FB82F96CC0863109F48EC075
:103DF00060F4813109F08CC00E943F1490910D0154
:103E000081E0892780930D0181C0893109F47EC04A
:103E10008B3109F07DC08091DB0181FB222720F9E5
:103E200091E0922790FB81F94CC0853309F466C07C
:103E300048F4873209F462C008F44FC0893209F4AB
:103E40005DC066C0833438F48A3308F044C08833D8
:103E500009F45CC05DC0833409F450C0883409F0B3
:103E600057C00E943F140FEF13ED20E301501040A4
:103E70002040E1F700C000000E94611B47C00E9483
:103E800053200E94A60F0E94A30840C09091DB011E
:103E9000892F8095817080FB90F929F09660986059
:103EA0009093DB0136C0997F977F9093DB012EC002
:103EB0008091DB0183FB222720F991E0922790FB80
:103EC00083F98093DB01992309F18091DB01816003
:103ED0008093DB011BC0895301C08D5141E050E04C
:103EE00060E070E08A019B0104C0000F111F221FD7
:103EF000331F8A95D2F7C901B80104C061E070E0B0
:103F000080E090E00E94FF170E943F1481E001C012
:103F100080E01F910F91089580E0089580E008955A
:103F20008E518A3030F4E82FF0E0E65DFE4F80815C
:103F3000089580E00895CF93C82F8091EB018130E0
:103F400079F018F08230E9F186C0E0910E01F0912D
:103F50000F018081813169F0823209F07EC009C091
:103F6000E0910E01F0910F018081813111F08232D8
:103F700061F48C2F0E948C1F811104C08C2F0E9431
:103F8000C91E1DC081E090E01AC08C2F0E948E1FB8
:103F9000811114C0C43179F048F4CB3079F0C031CC
:103FA00009F05FC082E08093EB0108C0C93219F0CC
:103FB000C83321F056C01092EB0153C081E08170EC
:103FC00052C0C93281F110F5C43169F1A8F4C7308B
:103FD00009F045C08AE08093150194E190931401A3
:103FE00093E0909313018093120188E08093110174
:103FF00088E28093100133C082EE8C0F863078F512
:104000008C2F0E94901F8093EA0129C0CE34E9F0E2
:1040100020F4CB3421F56AE013C0C13579F0C23504
:10402000F1F461E00DC08091EA01882319F010924B
:10403000EA0115C081E08093EB0115C061E006C084
:104040008091EA010E94031E0AC06AE08091EA01A1
:104050000E94791E04C01092EB0180E004C081E050
:1040600002C080E0ACCFCF910895E1E8F0E080811C
:10407000886080838081816080838FB7F89493E02B
:104080009093890090ED909388008FBF0895EFE69C
:10409000F0E08081826080830895EFE6F0E0808127
:1040A0008D7F80830895EFE6F0E0908182E089279C
:1040B000808308951F920F920FB60F9211242F93B1
:1040C0003F934F935F936F937F938F939F93AF93A0
:1040D000BF93EF93FF938091EC019091ED010196D6
:1040E0009093ED018093EC01811103C082E00E9466
:1040F000A308E091ED01E695E695F0E0EF59FC4F5D
:10410000E4918091EC018E1303C080E00E94A3082B
:10411000FF91EF91BF91AF919F918F917F916F919F
:104120005F914F913F912F910F900FBE0F901F9075
:10413000189504D06894B1118DC0089570D088F09E
:104140009F5790F0B92F9927B751A0F0D1F0660F83
:10415000771F881F991F1AF0BA95C9F712C0B1309E
:1041600081F077D0B1E0089574C0672F782F882749
:10417000B85F39F0B93FCCF3869577956795B395DD
:10418000D9F73EF490958095709561957F4F8F4F4C
:104190009F4F0895E89409C097FB3EF49095809551
:1041A000709561957F4F8F4F9F4F9923A9F0F92FFD
:1041B00096E9BB279395F695879577956795B7957B
:1041C000F111F8CFFAF4BB0F11F460FF1BC06F5F61
:1041D0007F4F8F4F9F4F16C0882311F096E911C073
:1041E000772321F09EE8872F762F05C0662371F094
:1041F00096E8862F70E060E02AF09A95660F771FA8
:10420000881FDAF7880F9695879597F9089557FDD7
:104210009058440F551F59F05F3F71F04795880F34
:1042200097FB991F61F09F3F79F0879508951216CB
:1042300013061406551FF2CF4695F1DF08C0161677
:1042400017061806991FF1CF869571056105089428
:104250000895E894BB2766277727CB0197F908953F
:104260000BD078C069D028F06ED018F0952309F0F3
:104270005AC05FC01124EECFCADFA0F3959FD1F3DF
:10428000950F50E0551F629FF001729FBB27F00D04
:10429000B11D639FAA27F00DB11DAA1F649F662759
:1042A000B00DA11D661F829F2227B00DA11D621FA8
:1042B000739FB00DA11D621F839FA00D611D221F62
:1042C000749F3327A00D611D231F849F600D211D46
:1042D000822F762F6A2F11249F5750408AF0E1F0E9
:1042E00088234AF0EE0FFF1FBB1F661F771F881F32
:1042F00091505040A9F79E3F510570F014C0AACFCD
:104300005F3FECF3983EDCF3869577956795B7951C
:10431000F795E7959F5FC1F7FE2B880F911D969546
:10432000879597F9089597F99F6780E870E060E0B6
:1043300008959FEF80EC089500240A94161617063E
:1043400018060906089500240A9412161306140686
:1043500005060895092E0394000C11F4882352F0E9
:10436000BB0F40F4BF2B11F460FF04C06F5F7F4FA1
:104370008F4F9F4F089597FB072E16F4009407D098
:1043800077FD09D00E94D52107FC05D03EF4909519
:1043900081959F4F0895709561957F4F0895EE0F19
:1043A000FF1F0590F491E02D0994AA1BBB1B51E15E
:1043B00007C0AA1FBB1FA617B70710F0A61BB70B95
:1043C000881F991F5A95A9F780959095BC01CD013A
:1043D0000895F999FECF92BD81BDF89A992780B5CD
:1043E0000895A8E1B0E042E050E00C941122262F9D
:1043F000F999FECF92BD81BDF89A019700B40216DB
:1044000039F01FBA20BD0FB6F894FA9AF99A0FBE88
:1044100008950196272F0E94F8210C94F721DC01C2
:10442000CB01FC01F999FECF06C0F2BDE1BDF89ABF
:10443000319600B40D9241505040B8F70895F89469
:02444000FFCFAC
:104442000220A50833091009DC08A8080101C801E7
:1044520028080A03140A404D36392103D4029E0269
:104462006502F80111022A02430201020304050651
:04447200070809002E
:00000001FF
